:1000000002308A00632A0000D3346D38EC32202A93
:10001000E832F236EF36653AE8327210A0060A008E
:10002000533A613B3A10253220147039EF3165376D
:10003000F430A9060A00533A613B3A1025266414AD
:100040007039EF316537F430A9060A00533A613B45
:100050003A10252664147039EF316537F430A9065B
:100060000A0083168611831286110830F80038289A
:100070000000F8174928F813B70C03188615031C5D
:100080008611781749287813F80B3C284728000078
:1000900086153F308400840B4B280000F81B3B285A
:1000A000781B43280800831603178C170C140000D4
:1000B000000083120C087F39031997280313AE0040
:1000C00003170D080313AF0003170F080313B00045
:1000D0002E08B70031202F0803178D0003133008B6
:1000E00003178F0083168C170C1400000000831276
:1000F0000C0D0E0D7F39031997280313AE0003175B
:100100000D080313AF0003170F080313B0002E08E8
:10011000B70031202F0803178D0003133008031791
:100120008F008D0A03198F0A031353280317031333
:100130008A110A12CB2A0830F800000086108316B4
:10014000861000008312AE0D0610031CAA28831629
:10015000061483120318AF28831606108312831621
:1001600086148312861CB228F80B9D280000861086
:100170008316861000000614000000008614831207
:10018000861CC028F8010000061878148610831613
:10019000861083120610831606108312080008309A
:1001A000AF007708B000831606140000861483128F
:1001B000861CD82806180314061C0310F80D00002E
:1001C0008316861083128610AF0BD328831606146D
:1001D00000008312061030080319F1288316061058
:1001E00083120000831686148312861CF5280000F3
:1001F00086108316861000008312061083160610E0
:1002000083120800831603178C170C1400000000DB
:100210000318312983120C087F390313B000031728
:100220000D080313B10003170F080313B2003008C1
:10023000B7003120310803178D000313320803176C
:100240008F0083168C170C14000000008312031318
:10025000AF0B2B292E29831603173129502983161A
:10026000031783120C0D0E0D7F390313B000031713
:100270000D080313B10003170F080313B200300871
:10028000B7003120310803178D000313320803171C
:100290008F008D0A03198F0A03100313AF0B022975
:1002A00008003608F8013502031859293508F70007
:1002B0006529F7010830B700B50DF70D360877024C
:1002C0000318F700F80DB70B5C2908002030301E2A
:1002D0003030B1002F08F700AF1F7529F709F70A72
:1002E0007708AF002D30B100B0172F08B50064308B
:1002F000B60051217708AF0030307807B2002F08E0
:10030000B5000A30B600512130307707B4003030E4
:100310007807B3003108F700B01D9029B01F3011E5
:10032000301A9D29B01FB8293019B8297708B200B2
:10033000B018B8297708B300B82930303202031D4D
:10034000B8297708B2002030B100B01DAB293011B8
:10035000B014B01FB01030303302031DB829770835
:10036000B3002030B200B01DAB29B010B01F301068
:10037000301DBD293108B7003120B01CC229320818
:10038000B7003120301CC7293308B70031203408AA
:10039000B70031208A110A12B22BB6010408B50049
:1003A0003610831B3614AF1FDD29B517351EB50A6D
:1003B000AE09AF09AE0A0319AF0A2F0EF038B1002B
:1003C000B107E23EB200323EB4002F080F39B20747
:1003D000B207B407E93EB300B307B3072E0E0F39D7
:1003E000B307B407B30DB40DB409B40D2E080F391B
:1003F000B407B10D0730B0000A30B407B303031CD3
:10040000FD29B307B203031C012AB207B103031C81
:10041000052AB107B003031C092A30308400831376
:1004200007303505351384033505031D1E2A351A9B
:10043000840A351A1E2A2030F7003B2A84073430FC
:100440000402031935170008F700031D2F2A351B76
:100450002F2A351A492AB5192F2A20303A2AB51FD2
:10046000372A2D30F70084033513B5133B2AB51511
:1004700035123030F707AF010408AE002F10831B90
:100480002F147708B70031202E08840083132F180B
:100490008317840A351F1F2A08002F308400831316
:1004A00000080319602A0230F800F701F70B562AFA
:1004B000F80B552A9730F700F70B5C2A800B532A6C
:1004C0008A110A12F72B840183131F3083057130C0
:1004D00083168F000F088611831286158316031763
:1004E0000908C039890003131F129F120030031737
:1004F00088008312870188018901FF300313A0005F
:10050000831603170908C039890003131F129F12AD
:10051000003003178800831203131F139F138316E1
:100520009F1383121F149412A012200883168700B1
:10053000831220162008831687008312A01120083A
:1005400083168700013083129400003083169400D4
:100550000108C73908388100831290010030F80083
:100560009200003083169200831220152008831613
:1005700087008312970183169B019C0101309D0027
:100580008312031787018801890104308D00003030
:100590008F0003135328A201A101A401A301831614
:1005A000061400008614000083120610831606103D
:1005B0000000831286108316861081308312AE00ED
:1005C0009B2078082D1078182D1483160610000033
:1005D00086148312861CEA2A0000EE2A0000831685
:1005E0000614000001308312AD06831606100000C9
:1005F00086148312861CFA2A0000FE2A0000831645
:100600000614000006140000861400008312061071
:100610008316061000008312861083168610803021
:100620008312AE009B20F330AE009B20831606148D
:100630000000861400008312861C1C2B06108316F3
:1006400006100000831286108316861081308312F4
:10065000AE009B20F701CF207808A800F701CF203B
:100660007808A70083160610000086148312861CE3
:10067000372B00003B2B00008316061400000614E5
:100680000000861400008312061083160610000076
:10069000831286108316861080308312AE009B2052
:1006A000F530AE009B20831606140000861400006F
:1006B0008312861C592B0610831606100000831225
:1006C00086108316861081308312AE009B20F701BE
:1006D000CF207808AA00F701CF207808A900831658
:1006E0000610000086148312861C742B0000782BE1
:1006F00000008316061400008312AF012808AE0024
:10070000AF00AE012708AE070318AF0A2F0CA200F6
:100710002E0CA100A20CA10C3F30A205AF012A08AB
:10072000AE00AF00AE012908AE070318AF0A2F0CC8
:10073000A4002E0CA300A40CA30C3F30A405003091
:100740002D180130AE00103003178D0000308F00DF
:10075000031006300313AF0002212E08AF001F3034
:10076000B0006629143003178D0000308F0003108D
:100770000D300313AF0002211B3003178D00003032
:100780008F00031006300313AF00022110308400E5
:100790002208AF002108AE00CD211F3003178D00C5
:1007A00000308F0003140C300313AF0002212630F9
:1007B00003178D0000308F00031006300313AF00C5
:1007C0000221103084002408AF002308AE00CD21A0
:1007D0002A3003178D0000308F0003140C300313F0
:1007E000AF0002210830AE00FA30AF004D2AAE0B48
:0607F000F42BCB2A63008C
:04400E00F52CFF3F4F
:00000001FF
